:100000000C94B3020C94EB020C94EB020C94EB02F4
:100010000C94EB020C94EB020C94EB020C94EB02AC
:100020000C94EB020C94EB020C94EB020C94252A3A
:100030000C94D42A0C9437250C94EB020C94EB020C
:100040000C94EB020C94EB020C94781F0C94BF25DB
:100050000C94EB020C94EB020C94EB020C94EB026C
:100060000C94EB020C94EB020C94EB020C94EB025C
:100070000C94EB02C405C405F005F005580676069D
:100080008E078E0781061A072B072B07851E871EF2
:100090008C1E8F1E921E951E981E412237224422CE
:1000A0008C22902290228C229022902265229022F3
:1000B0006F22792290229022902290228C229022EC
:1000C00090228C22902252229022902289228922F0
:1000D00089228922892289228922892289228E22C3
:1000E000902241223422902290229022902290222B
:1000F000902290229022902290228E229022902272
:100100008C22902287228722872287228722872299
:100110008722872287228E22412B682B602C682B16
:10012000602CB42BD72B602C2E2C3D2C2900E0000A
:10013000E2002A0053005400550056005F006000A2
:10014000610057005C005D005E00570059005A00D6
:100150005B005800620062006300580000047F3FAB
:100160001F643214643214783C1E1E140A052223C4
:10017000252628292A2C2D2F3032333536383A3B84
:100180003D3E4042434547494A4C4E5051535557D6
:10019000595A5C5E6062646668696B6D6F717375F5
:1001A00077797B7D7F81838587898A8C8E909294F5
:1001B00096989A9C9E9FA1A3A5A7A8AAACAEAFB102
:1001C000B3B4B6B8B9BBBCBEBFC1C2C3C5C6C7C94C
:1001D000CACBCCCDCED0D1D2D2D3D4D5D6D7D7D806
:1001E000D9D9DADADBDBDBDCDCDCDCDCDDDDDDDD58
:1001F000DCDCDCDCDCDBDBDBDADAD9D9D8D7D7D660
:10020000D5D4D3D2D2D1D0CECDCCCBCAC9C7C6C516
:10021000C3C2C1BFBEBCBBB9B8B6B4B3B1AFAEAC5C
:10022000AAA8A7A5A3A19F9E9C9A98969492908E07
:100230008C8A89878583817F7D7B79777573716FE0
:100240006D6B6968666462605E5C5A5957555351BC
:10025000504E4C4A4947454342403E3D3B3A383672
:10026000353332302F2D2C2A292826252322FFAA88
:100270007F55400000000000000000000000010168
:100280000203040506080A0C0F1114181C20242967
:100290002E33393F464C535B626A7179818A929A58
:1002A000A2AAB2B9C1C8CFD5DCE1E7EBF0F4F7FA06
:1002B000FCFDFEFFFEFDFCFAF7F4F0EBE7E1DCD518
:1002C000CFC8C1B9B2AAA29A928A8179716A625BD7
:1002D000534C463F39332E2924201C1814110F0C7F
:1002E0000A080605040302010100000000000000E6
:1002F00000000000010101010101010101020202EF
:1003000002020202020203030303030303030404C1
:10031000040404040405050505050606060606078B
:100320000707070708080808090909090A0A0A0B44
:100330000B0B0C0C0C0D0D0D0E0E0E0F0F0F1010E5
:10034000111111121213131414151516161717186C
:100350001819191A1A1B1B1C1D1D1E1E1F202021D7
:100360002222232424252626272829292A2B2C2D1E
:100370002D2E2F30313232333435363738393A3B3F
:100380003C3D3E3F404142434445464748494A4C34
:100390004D4E4F50515354555658595A5B5D5E5F00
:1003A000616264656668696B6C6D6F707273757796
:1003B000787A7B7D7E8082838587888A8C8E8F91F8
:1003C000939596989A9C9EA0A2A3A5A7A9ABADAF22
:1003D000B1B3B5B7BABCBEC0C2C4C6C9CBCDCFD10C
:1003E000D4D6D8DBDDDFE2E4E7E9EBEEF0F3F5F8B5
:1003F000FAFDFF18034B0042004400500041004446
:10040000002D004D004B0049004900000010034B37
:100410000042004400660061006E007300000004AA
:1004200003090409023B00020100A0FA09040000CC
:10043000010301010009211101000122400007050B
:1004400081030800010904010001030000000921E3
:100450001101000122B600070582032000011201EC
:1004600000020000000803A10600010001020001D3
:1004700005010902A10185020901A100050919016F
:10048000290815002501950875018102050109302B
:1004900009311581257F9502750881060938158176
:1004A000257F950175088106050C0A3802158125FE
:1004B0007F950175088106C0C005010980A10185ED
:1004C0000319012AB700150126B70095017510819F
:1004D00000C0050C0901A101850419012AA002151B
:1004E0000126A002950175108100C005010906A131
:1004F000018506050719E029E7150025019508750E
:100500000181020507190029EF1500250195F075F5
:1005100001810205081901290595057501910295CA
:100520000175039101C005010906A101050719E044
:1005300029E71500250195087501810295017508C7
:1005400081010507190029FF150026FF0095067592
:100550000881000508190129059505750191029585
:100560000175039101C011241FBECFEFD4E0DEBF9F
:10057000CDBF04B603FE18C0809111039091120301
:10058000A0911303B09114038730904BA740B04B58
:1005900059F4109211031092120310921303109247
:1005A0001403E0E0F8E3099511E0A0E0B1E0E6EF24
:1005B000FAE502C005900D92A03CB107D9F723E0FF
:1005C000A0ECB1E001C01D92A131B207E1F70E9499
:1005D00078130C94792D0C94000081E0089581E04B
:1005E00008950C94EF0208950C94F3021F93CF9397
:1005F000DF9300D000D01F92CDB7DEB749835A8376
:100600006B833091C30189819A81311114C06623B3
:1006100059F0222349F00E94CE09182F682F8981B2
:100620009A810E94740903C00E94A209182F69814F
:100630007A81812F04C00E94CE0969817A810F904E
:100640000F900F900F900F90DF91CF911F910C940E
:10065000F510FC01262F40815181628173818481D4
:100660000C94F60281E00895CF93DF93EC0160E0F3
:100670000E942903BE01DF91CF910C94F4020C94E7
:100680003B120C94371208950E941E080E944303E7
:100690002FEF84E39CE0215080409040E1F700C0C0
:1006A00000000C94E5250F931F93CF93DF938C01EB
:1006B00061E00E942903EC01B8010E94F102882345
:1006C00009F44BC0B801CE010E94761E882309F4BC
:1006D00044C0B801CE010E9483238823F1F1B80100
:1006E000CE010E9447208823C1F1B801CE010E94AB
:1006F000DF22882391F1B801CE010E948D1C88234E
:1007000061F1F8018281882309F1CB358DE5D807A5
:10071000C1F050F4C115FCE5DF0781F0CF3DDC45A9
:10072000A9F40E94010F19C0CC35EDE5DE0761F098
:10073000CD35DD4559F40E94440E08C00E944403A3
:100740000CC00E944D0E02C00E94500EC801DF91E5
:10075000CF911F910F910C94ED0280E0DF91CF912A
:100760001F910F9108950E941A2580E00E942C1F6E
:100770000E94E2030C940A1B0E949A1D0E94E5034A
:100780000E94D61B0C94202508950C94C40381E08C
:100790000895CF93C82F0E94C703882329F0C0FD76
:1007A00002C02C9A01C02C98CF910895249A2C9ABB
:1007B0000895CF93C82F0E94C5038C2F0E94C903B0
:1007C000CF91089580E00C94D9030E94DF230C940C
:1007D000D9030E94DF239091C201891721F08093F1
:1007E000C2010C94D9030895CF93DF93CDB7DEB740
:1007F0002B970FB6F894DEBF0FBECDBF4F8358873F
:1008000069877A878B8761110E94900D9E012F5F07
:100810003F4F86E0F90111928A95E9F785E0FE01E4
:100820003796D90101900D928A95E1F789819A81D5
:100830004C815D81452B31F09F3F31F491E08F3F3A
:1008400019F403C091E001C090E090FF09C0498114
:100850005A816B817C818D819E810E94AC0C05C088
:10086000C9010E9432038111F2CF2B960FB6F89482
:10087000DEBF0FBECDBFDF91CF910895FC01808117
:1008800091810E94100A0895CF93882309F4A9C08A
:10089000C82F8238C1F40E94DF2381FDA2C069E322
:1008A00080910201909103010E94D5240E94B20D13
:1008B0002FEF81EE94E0215080409040E1F700C09E
:1008C000000069E319C0833801F50E94DF2380FD31
:1008D00088C063E580910201909103010E94D524B4
:1008E0000E94B20D2FEF81EE94E0215080409040A5
:1008F000E1F700C0000063E58091020190910301DF
:100900000E94E024CF910C94B20D8438C1F40E946F
:10091000DF2382FD66C067E48091020190910301AC
:100920000E94D5240E94B20D2FEF81EE94E0215059
:1009300080409040E1F700C0000067E4DDCF8CEF1D
:100940008C0F813AF8F48C2F0E949622811149C0B5
:100950006C2F80910201909103010E9455248823FD
:1009600049F06C2F80910201909103010E94E024D4
:100970000E94B20D6C2F80910201909103010E94A0
:10098000D524C0CF80E28C0F883048F4C77081E056
:1009900001C0880FCA95EAF70E94730DB3CFEBE54B
:1009A000EC0FE33040F4F0E0E45AFE4F808190E039
:1009B000CF910C941324E8E5EC0FE73150F4F0E00C
:1009C000EE0FFF1FE25DFE4F80819181CF910C946D
:1009D0002924CD3E30F08C2F0E940514CF910C9429
:1009E000D714CF910895882309F464C0823879F42C
:1009F0000E94DF2381FF5EC069E380910201909134
:100A000003010E94D5240E94B20D69E310C083380F
:100A1000B1F40E94DF2380FF4DC063E580910201A5
:100A2000909103010E94D5240E94B20D63E580914C
:100A30000201909103010E94E0240C94B20D8438CD
:100A400079F40E94DF2382FF35C067E480910201C0
:100A5000909103010E94D5240E94B20D67E4E7CF74
:100A60009CEF980F913A10F4682FE1CF90E2980F25
:100A7000983050F4877091E001C0990F8A95EAF799
:100A8000892F0E94790DD9CF9BE5980F933020F4E0
:100A900080E090E00C94132498E5980F973120F4AF
:100AA00080E090E00C9429248D3E20F00E94601498
:100AB0000C94D71408951F93CF93DF93182FEB0155
:100AC0000E944404209741F08FE99FE00197F1F7DD
:100AD00000C000002197F6CF812FDF91CF911F91A9
:100AE0000C94F304893319F060E070E002C060E513
:100AF00070E00C945B05882321F00E94730D0C9428
:100B0000B20D0895882321F00E94790D0C94B20D46
:100B10000895CF92DF92EF92FF920F931F93CF939E
:100B2000DF937C01D62FC72FFC011281058102952E
:100B30000F700E94690D8823B9F01123A9F08C2F42
:100B4000807F803421F080E28D0F883068F08091C2
:100B5000BD0282FD09C082E00E94120E0E94690D52
:100B600091E0D82ED92601C0D12CCC2EC2948FE092
:100B7000C8228C2D90E08C30910508F0CFC1FC018B
:100B8000E65CFF4F0C94112D8C2F807FCF70882353
:100B900011F0C295C07F112399F0CC2309F4AAC1AA
:100BA00080E28D0F883010F0D11104C08C2F0E948C
:100BB000730D03C08C2F0E94830D0E94B20D9AC149
:100BC0008D2F0E94F304CC2309F4A8C180E28D0F7D
:100BD000883038F1DD2329F18C2F0E94890D24C043
:100BE0008C2F807FCF70803211F0C295C07FDD23C3
:100BF00019F0D130A1F13DC08091BD0282FF17C034
:100C0000112349F0CC2329F08C2F0E94730D0E94F0
:100C1000B20D80E070C180E00E94F304CC2309F49F
:100C20007DC18C2F0E94790D0E94B20D77C11123D6
:100C300071F0002341F0013031F40E94930D8C2BB0
:100C40000E949B0D6BC10E94930D8C2B1DC0002335
:100C500019F0013009F462C10E94A80D25C01123CA
:100C600021F0063008F05AC10EC0053008F056C118
:100C70001BC0112361F0002331F0F701858180FF53
:100C800039C18F7085838C2F0E947B0547C100235B
:100C900059F0D93309F03FC1FFEF07EE13E0F150EF
:100CA00000401040E1F735C18C2F0E94820536C10B
:100CB0008C2F86958695837019F0813061F02EC156
:100CC000112321F08D2F9C2F937002C080E090E0C3
:100CD0000E9413242BC1112321F08D2F9C2F937080
:100CE00002C080E090E00E94292420C18D2F1123B2
:100CF00019F00E94051402C00E9460140E94D714CB
:100D000015C18C2F837009F047C011110BC12D2F15
:100D1000229526952770220F220F6D2F6F70862F38
:100D200090E0A0E0B0E0022E04C0880F991FAA1F37
:100D3000BB1F0A94D2F7D4FF10C04FE050E060E030
:100D400070E004C0440F551F661F771F2A95D2F725
:100D5000409550956095709503C040E050E0BA0111
:100D6000C695C695C3708A019B01082B192B2A2BA7
:100D70003B2BC901B801C23049F058F4C13019F019
:100D80000E948A08CFC00E947808CCC00E949C08AC
:100D9000C9C00E947608C6C0112319F08C2F81703B
:100DA00001C08695882309F4BDC02D2F2295269574
:100DB0002770220F220F6D2F6F70862F90E0A0E01A
:100DC000B0E0022E04C0880F991FAA1FBB1F0A940F
:100DD000D2F7D4FF10C04FE050E060E070E004C0F4
:100DE000440F551F661F771F2A95D2F740955095DF
:100DF0006095709503C040E050E0BA01C695C69575
:100E0000C3708A019B01082B192B2A2B3B2BC9018C
:100E1000B801C23049F058F4C13019F00E944F09AE
:100E200081C00E943D097EC00E9461097BC00E9472
:100E3000B00878C0CF70112339F08C2F0E94D608EB
:100E40008D2F0E947B056EC08D2F0E9482058C2FF6
:100E50000E94F70867C0D23F21F128F4D03F41F04B
:100E6000D13FC1F043C0D33F19F1D43F79F03EC028
:100E7000112341F0053008F051C08C2F8F710E9472
:100E80001C094CC0063008F049C0F7CF8091BD0264
:100E900082FF18C0112339F08C2F8F710E94D60861
:100EA0003DC01123C9F38C2F8F710E94F70836C003
:100EB000112329F08C2F8F710E94C1082FC00E942E
:100EC000BC082CC0112349F0CF718C2F0E94D6088A
:100ED00063E08C2F0E94F70D21C081E00E94120E6A
:100EE0000230E0F082E00E94120E18C0112331F0AF
:100EF000002391F28D2F0E94440410C0002399F228
:100F0000D93349F41FEF27EE33E011502040304031
:100F1000E1F700C000008D2F0E94F30488EF8C0DD4
:100F2000843020F40E94DF230E94D903DD20C9F021
:100F30000E94650D80FD15C0F70112820E945F0DB1
:100F40000E94D608C7010E94D2070E945F0DDF9160
:100F5000CF911F910F91FF90EF90DF90CF900C9465
:100F6000F708DF91CF911F910F91FF90EF90DF90E5
:100F7000CF9008950F931F93CF93DF93EC01688177
:100F800079818A810E941B0A8C010E9473090E9448
:100F90006408B801CE010E948905DF91CF911F91AD
:100FA0000F910895CF93DF93EC01988189812B8174
:100FB0003C81232B31F08F3F31F481E09F3F19F4C6
:100FC00003C081E001C080E080FD1DC0CE010E9411
:100FD0005303811110C00E94690D8823A1F08A81FA
:100FE000882389F08091BD0282FD0DC082E0DF91EF
:100FF000CF910C94120ECE010E94BA07CE01DF9160
:10100000CF910C943403DF91CF91089580E090E06C
:101010000E94132480E090E00E9429240E94900DF9
:101020000E94B20D0E9416160C94D71480910201F2
:10103000909103010E94EB240C9406080E94800DFD
:101040000C94160892959F70963079F010F4925097
:1010500001C09A50923068F4803F69F018F4883EDD
:1010600040F409C0843F29F406C0883E20F0813F47
:1010700011F080E0089581E00895FC018081918164
:101080000E94100A0E9422080895CF93DF9300D097
:1010900000D01F92CDB7DEB70F900F900F900F903A
:1010A0000F90DF91CF910895CF93DF9300D000D0C0
:1010B00000D0CDB7DEB726960FB6F894DEBF0FBED0
:1010C000CDBFDF91CF910895089508950C946508E0
:1010D0000C9466080E9468086093D7017093D80149
:1010E0008093D9019093DA010C9406080C946A0855
:1010F0000F931F930091D7011091D8012091D9012E
:101100003091DA01602B712B822B932B1F910F9161
:101110000C946A080F931F930091D7011091D80186
:101120002091D9013091DA01602371238223932326
:101130001F910F910C946A080F931F930091D70190
:101140001091D8012091D9013091DA0160277127DF
:10115000822793271F910F910C946A080C946508BD
:101160000E94AE086093D3017093D4018093D5019F
:101170009093D6010C94060860E070E0CB010C94CB
:10118000B0080F931F9341E050E060E070E08A01E7
:101190009B0104C0000F111F221F331F8A95D2F735
:1011A000C901B8011F910F910C94B0080F931F93C0
:1011B00041E050E060E070E004C0440F551F661F3E
:1011C000771F8A95D2F78091D3019091D401A09195
:1011D000D501B091D6018A019B01082B192B2A2B2E
:1011E0003B2BC901B8011F910F910C94B0080F93CC
:1011F0001F9341E050E060E070E004C0440F551FD1
:10120000661F771F8A95D2F7409550956095709527
:101210008091D3019091D401A091D501B091D601D4
:101220008A019B01082319232A233B23C901B80102
:101230001F910F910C94B0080F931F9341E050E061
:1012400060E070E004C0440F551F661F771F8A9549
:10125000D2F78091D3019091D401A091D501B091A2
:10126000D6018A019B01082719272A273B27C90194
:10127000B8011F910F910C94B0080F931F93009128
:10128000D3011091D4012091D5013091D601602B6A
:10129000712B822B932B1F910F910C94B0080F93FD
:1012A0001F930091D3011091D4012091D501309169
:1012B000D60160237123822393231F910F910C94F5
:1012C000B0080F931F930091D3011091D401209186
:1012D000D5013091D60160277127822793271F916E
:1012E0000F910C94B0080895262F990F990F890F2C
:1012F000982F9770A1E001C0AA0F9A95EAF78695FA
:101300008695869590E065E070E00E949D2CFC013A
:10131000EC53FE4F40E050E0622F70E090819B0163
:10132000042E02C0369527950A94E2F72170219584
:1013300029272A23292721934F5F5F4F45305105E5
:1013400069F70895990F990F890FA82FA7708695AF
:101350008695869590E065E070E00E949D2CBC012A
:1013600040E050E080E0FB01E40FF51FEC53FE4F3E
:10137000208130E00A2E02C0369527950A94E2F7C4
:1013800021703327042E01C0220F0A94EAF7822B22
:101390004F5F5F4F4530510531F70895BF92CF92AF
:1013A000DF92EF92FF920F931F93CF93DF938C0105
:1013B000C090D301D090D401E090D501F090D60137
:1013C0008091D7019091D801A091D901B091DA0113
:1013D000C82AD92AEA2AFB2ACFE1D0E0D701C601E0
:1013E0000C2E04C0B695A795979587950A94D2F7C9
:1013F00080FD04C0219790F7B12C07C0BC2EB80126
:101400008C2F0E940B110197A9F38B2DDF91CF91A7
:101410001F910F91FF90EF90DF90CF90BF900895B4
:10142000CF93DF93EC010E94CE09BE010E940B1105
:10143000DF91CF9108951F93CF93DF93EB019091AC
:10144000C301992321F0CB010E94100A13C0882305
:1014500049F0CB010E94CE09182F682FCE010E94BF
:10146000740904C0CB010E94A209182FBE01812F6C
:101470000E940B11DF91CF911F910895CF93DF93BD
:10148000C091DB018091DC01C817A1F0D0E0CE0152
:1014900066E070E00E949D2CFC01E352FE4F40810B
:1014A000518162817381848195810E9454082196C3
:1014B000C770E8CFDF91CF91089540910D02509110
:1014C0000E0260910F0270911002809111029091B2
:1014D00012020C945408FF920F931F93CF93DF9343
:1014E0008091120282958F7009F062C080910F0284
:1014F000882309F45DC02091DB01F090DC0110919C
:101500000D0200910E02A0911002B091110281E033
:101510001F3F09F080E0C0910001D0910101482FE8
:101520002F1509F445C0109721F00F3F21F080E0FE
:1015300003C081E001C0842F30E080FD35C0C901C7
:1015400066E070E00E949D2CFC01E352FE4F818119
:1015500080132AC08081811327C08281811124C019
:10156000838194818A1B9B0B8C179D07E8F48091E3
:1015700012028F70806180931202C90166E070E0F0
:101580000E949D2CFC01EE51FE4F90819F70906156
:1015900090838DE092E00E94D207DF91CF911F915E
:1015A0000F91FF900C943E0A2F5F3F4F2770B8CFEA
:1015B000DF91CF911F910F91FF9008959F92AF926D
:1015C000BF92CF92DF92EF92FF920F931F93CF9330
:1015D000DF93CDB7DEB761970FB6F894DEBF0FBECD
:1015E000CDBF8C0185E0F801DE011D9601900D92C2
:1015F0008A95E1F7F801E28090910D0230910E0298
:1016000060911002709111026115710531F03F3F38
:1016100031F481E09F3F19F403C081E001C080E014
:10162000F82FF1709F2E80FD47C1F8014081218184
:10163000A380B4808DE0C82E82E0D82EF0900F02F7
:10164000F501E61BF70B6091000170910101FF208D
:1016500009F4DCC080911202582F507FE617F7077B
:1016600008F096C0511155C0231313C0491311C07F
:10167000FE2CE1100EC08F708061809312020E94D8
:101680005D0AC6010E94D20780911202F80185838B
:1016900050C1AB2831F02F3F31F481E04F3F19F4B6
:1016A00003C081E001C080E080FD03C081E08E25A1
:1016B00002C080E090E0F82FF170FF2E80FF1FC085
:1016C000E091DB013091DC01E31709F410C1F0E097
:1016D000CF0166E070E00E949D2CDC01A352BE4F5A
:1016E00011968C911197281307C08C91481304C050
:1016F00012968C91E81203C03196E770E5CFFE2C6C
:10170000EE2009F416C180911202816080931202CA
:1017100054C0231306C0491304C0E11002C0F801ED
:1017200099C0C8010E943D08882361F1EE2051F163
:1017300020911202822F82958F7090E0029774F0B0
:1017400080910D0290910E0298878F831986BB8637
:10175000AA862C87CE0107960E94D20786E0F80160
:10176000ADE0B2E001900D928A95E1F70E946B0A1C
:101770000E945D0A0AC0231711F1C8010E943D08AA
:1017800081112CC0C8010E94D207FF24F394D1C05C
:101790005111F1CF7A2DB98AA88A522F6E2D8989DD
:1017A0000E9445088DE092E00E94D20786E0F60193
:1017B00011928A95E9F70E945D0AF12CBAC049138B
:1017C000DCCFE110DACFF8018583C8010E94D2078F
:1017D00086E0F60111928A95E9F7ABC0EE2091F20E
:1017E00020911202822F82958F7090E002970CF464
:1017F000B5CF80910D0290910E029A8389831B824E
:10180000BD82AC822E83CE010196A6CFE617F707E4
:1018100008F044C0FE2CEE2009F4B4CF231330C0EE
:1018200049132EC02091120220FD21C0822F8295E3
:101830008F70482F50E041155105C9F0F8012583FC
:101840004F30510541F08F5F982F9295907F822FF6
:101850008F70892B8583C8010E94D20786E0F8012A
:10186000ADE0B2E001900D928A95E1F73DC086E0CF
:10187000F801ADE0B2E001900D928A95E1F759C010
:10188000C8010E943D08811169CF809112028160D8
:1018900080931202C8010E94D2074BC07A2DB98AE8
:1018A000A88A522F6E2D89890E94450886E0F6018C
:1018B00011928A95E9F718C0EE2009F463CFC801A8
:1018C0000E943D08F82E882309F45CCF86E0F801D9
:1018D000ADE0B2E001900D928A95E1F78DE092E0E3
:1018E0000E943E040E946B0A0E945D0A22C04D873E
:1018F0002E878D859E850E94100A292F22952F7094
:10190000223028F49F7039F0811105C00BC02430BB
:1019100028F49F7049F4805E883020F0C8010E944E
:10192000D2079F2CF92C05C0F8019581907F99F77B
:10193000F9CF8F2D61960FB6F894DEBF0FBECDBFE5
:10194000DF91CF911F910F91FF90EF90DF90CF909B
:10195000BF90AF909F900895CF93DF93CDB7DEB740
:101960002C970FB6F894DEBF0FBECDBF4F835887BC
:1019700069877A878B879C87CE0107960E94DE0A4B
:101980008823D1F09F8188852A853B85232B31F0E0
:101990008F3F31F481E09F3F19F403C081E001C023
:1019A00080E080FD6FC04F81588569857A858B8581
:1019B0009C850E94540866C086E0FE013796DE01D1
:1019C000119601900D928A95E1F7FF81E8856A856D
:1019D0007B856115710531F0EF3F31F481E0FF3F08
:1019E00019F403C081E001C080E080FD4BC080910C
:1019F000DC0190E09C012F5F3F4F2770332740911F
:101A0000DB0150E02417350709F443C0F983EA836A
:101A10007D836C8366E070E00E949D2CDC01A35204
:101A2000BE4F96E0FE01319601900D929A95E1F736
:101A30002093DC010E943E0A25C090E066E070E041
:101A40000E949D2C83529E4F0E94DE0A882371F1D2
:101A50008091DB0190E066E070E00E949D2CFC012B
:101A6000E352FE4F4081518162817381848195816F
:101A70000E9454088091DB0190E0019687709927BD
:101A80008093DB018091DB019091DC018913D5CF3C
:101A90000DC00E941E081092DC011092DB01EDE0E7
:101AA000F2E086E0DF011D928A95E9F72C960FB6E9
:101AB000F894DEBF0FBECDBFDF91CF910895809126
:101AC00033028595859585950895809133028770B9
:101AD000089590913302977081E009F480E00895B1
:101AE00080915602089590915602892B8093560258
:101AF0000895809590915602892380935602089507
:101B000010925602089590915502892B80935502A8
:101B100008958095909155028923809355020895E8
:101B200010925502089580913402089508950C94FE
:101B3000960D0C94970D9091BD0292FD08C0909166
:101B40003402981721F0809334020C94990D089573
:101B500080913402882329F01092340280E00C94A2
:101B6000990D0895CF93DF93E0910201F091030165
:101B7000809156028083E0910201F09103019081EF
:101B800080915502892B808380913402882381F0D3
:101B9000E0910201F09103019081892B8083809173
:101BA0000201909103010E943F2481110E94A80D1F
:101BB000C0910201D091030140E250E063E172E084
:101BC000CE010E94242D892B69F080E2FE01A3E161
:101BD000B2E001900D928A95E1F7CE01DF91CF91AD
:101BE0000C94EB23DF91CF9108950C94960D909176
:101BF000BD0292FD10C0982F990F990F990F692B74
:101C0000609333020E94D6088091330285958595B2
:101C100085950C94F50D0C94D6081092330280E053
:101C20000C94F50D2091330280958223809333022A
:101C3000982F977099F430E0482F082E000C550B20
:101C40002417350759F09091BD0292FD07C0859584
:101C5000859585950E94F7080C940D0E0895909136
:101C6000BD0292FB222720F9281769F080FB92F928
:101C70009093BD028091BC029091BD020E947D0EA6
:101C800082E00C94120E08958091BD0282FB882799
:101C900080F991E089270C942F0E81E00C942F0E8F
:101CA00080E00C942F0E6FEF7FEF80E090E00C94BB
:101CB000632D80E090E00E943F2D21E0893E9E4F01
:101CC00009F020E0822F089582E090E00C94312DFD
:101CD00083E090E00C94312DCF9384E090E00E945B
:101CE000312DC82F82E290E00E94312D2C2F30E060
:101CF000A901582BCA01CF910895CF93C92F682FFE
:101D000084E090E00E94452D6C2F82E290E0CF911C
:101D10000C94452DAB01BC018FE090E00C94572D45
:101D2000AB01BC0183E190E00C94572D60E070E0C2
:101D3000CB010C94900E60E070E0CB010E948A0E03
:101D40000C94960E69EE7EEF80E090E00E94632D89
:101D500060E082E090E00E94452D60E083E090E04A
:101D60000E94452D1092D7011092D8011092D901EE
:101D70001092DA0160E084E090E00E94452D60E07E
:101D800082E290E00E94452D60E085E090E00E94B4
:101D9000452D60E086E090E00E94452D6FEF87E0E2
:101DA00090E00E94452D40E050E0BA0188E090E0CC
:101DB0000E94572D60E08DE090E00E94452D40E0AC
:101DC00050E0BA0188E190E00E94572D60E087E181
:101DD00090E00E94452D40E050E0BA018CE190E097
:101DE0000E94572D60E070E080E290E00E94632D39
:101DF00040E050E0BA0188E190E00E94572D0C9439
:101E00009B0E0C94A20E682F8EE090E00C94452D52
:101E10000E94A42560936102709362028093630222
:101E20009093640260935D0270935E0280935F0200
:101E300090936002089581E008950C941B0F08951B
:101E40000C941F0F0C941F0F0C94220F0C941F0F57
:101E50000C94260F0C941F0F87EE91E10E94D5235E
:101E60000E942A0F0C94280F0E94200F0C941F0F21
:101E70000E9401120E94D6030C9406200E948F2516
:101E80000E94D8120E94380F0E949A1D0E949B1B2C
:101E90000C94240F8F929F92AF92BF92CF92DF92B9
:101EA000EF92FF920F931F93CF93DF93CDB7DEB7DF
:101EB0002A970FB6F894DEBF0FBECDBF0E94ED1279
:101EC000982E81110E94080F87E5A82E82E0B82E77
:101ED00000E010E0802E802F0E942512D82EF50100
:101EE000C1905F01C826B1F40F5F1F4F0630110586
:101EF00089F78FEF89838A831B820E9498258160EE
:101F0000782F9D838C8349815A816B818D810E94BA
:101F1000F4032FC08091650281FD0E942B12E12CF9
:101F2000FF24F3948C2D8F21F1F00E941D0F882344
:101F300099F0EE828F82DF2081E009F480E08887CB
:101F40000E9498258160782F9A8789874E815F81CA
:101F500068858A850E94F403F801E95AFD4F808163
:101F6000F826F08206C0E394FF0CF4E0EF12DACF1B
:101F7000BBCF81E0911001C080E02A960FB6F894A3
:101F8000DEBF0FBECDBFDF91CF911F910F91FF90AC
:101F9000EF90DF90CF90BF90AF909F908F9008957B
:101FA0000E944A0F0E94DF1B0E94621F0E94F514CC
:101FB0000C94E903CF93DF930E941011EC0181157B
:101FC00021E5920708F045C0811530E5930708F038
:101FD00094C0883E910528F5803E910508F001C126
:101FE000883A910570F4853A910508F07CC08130FB
:101FF000910509F475C008F4F1C0049708F0F1C028
:10200000EDC08F3B910508F0E9C0C85AD0E0CC0F75
:10201000DD1FC15ADE4F0990D881C02DCE019464D6
:10202000E1C0811540E2940758F4811551E095070D
:1020300008F0D7C08D3E910508F4D0C09065D2C09D
:10204000C11580E4D80708F4C9C0DF70CE01906ADA
:10205000C9C0811525E59207A8F4811534E59307D9
:1020600008F09EC0811543E5940708F081C08115F2
:1020700052E5950708F064C0D82FCC27CE01816FB8
:10208000906AB0C0C11589E5D807A0F4C11528E54C
:10209000D20708F08BC0C11536E5D30708F09EC003
:1020A0008C2F0E94A4118F7190E0D82FCC27CE01E5
:1020B000906298C0C1154AE5D40708F47DC0CE01EE
:1020C00090568115904208F089C08D2F8F710E9423
:1020D000A411DD27D0628F71AE01582BCA0182C0D6
:1020E00081E090E07FC0C55AD0E0C357DE4F8881C1
:1020F000C82FD0E0CE01906475C0F4E09695879526
:10210000FA95E1F7282F23703C2F337081E090E09F
:1021100002C0880F991F3A95E2F79C68AC01522BD8
:102120009C2F9F7096959695892F90E0EC01A5E0E5
:10213000CC0FDD1FAA95E1F7CA018C2B9D2B52C055
:102140008370992721E030E002C0220F331F8A9567
:10215000E2F79C2F96959695C92FD0E075E0CC0FAD
:10216000DD1F7A95E1F7C22BD32BCE019C683AC0D4
:102170008370992721E030E002C0220F331F8A9537
:10218000E2F79C2F96959695C92FD0E065E0CC0F8D
:10219000DD1F6A95E1F7C22BD32BCE019A6822C0CE
:1021A000D82FCC27CE01846F906A1CC0DC2FCC279F
:1021B000CE01806F906A16C08C2F8F700E94A41180
:1021C00094E0D695C7959A95E1F7CF70D0E0DC2FD3
:1021D000CC27D0699E01282BC90104C080E090E083
:1021E00001C0CE01DF91CF9108959B0190E066E0A0
:1021F00070E00E949D2C830F911DFC01EE0FFF1FCC
:10220000EE0FFF1FE20FF11DEE0FFF1FE45DFE4F0B
:102210008591949108950E94F5100E94DA0F089517
:102220008238910569F1B0F48133910509F46DC0EC
:1022300048F48932910509F463C08A32910509F4A2
:1022400069C008958533910509F455C08933910516
:10225000B9F00895833E910569F138F4803E910507
:10226000B1F0823E910509F10895863E9105A9F1EC
:10227000873E9105B9F1843E910509F064C023C001
:102280002091BC0220FD4FC021FD4DC008958091DA
:10229000BC0280FD44C08091BD0280FF44C080919B
:1022A000BC0284FD42C083EE4DC08091BC0282FF1F
:1022B00038C0F5CF8091BC0282FD33C08091BD0251
:1022C00080FD31C0ECCF8091BD0281FF32C0809192
:1022D000BC0284FD2AC087EE35C08091BC0283FF1A
:1022E00026C0F5CF8091BC0283FD21C08091BD0244
:1022F00081FD1FC0ECCF8091BC0285FD1CC01DC0BC
:102300008091BC0285FD19C016C08091BC0286FD7B
:1023100016C017C08091BC0286FD13C010C089E3AF
:1023200011C082EE0FC080EE0DC080E00BC086EEC3
:1023300009C084EE07C089E205C085E303C08AE2D4
:1023400001C081E390E008959091BC0292FF0DC01E
:10235000282F2871283019F4877F846006C0282F21
:102360002471243011F48B7F886093FF0DC0282FD7
:102370002871283119F4877E846106C0282F2471C2
:10238000243111F48B7E88612091BD0220FF0DC0A5
:10239000382F3871383019F4877F816006C0382FA4
:1023A0003171313011F48E7F886021FF0DC0282FEC
:1023B0002871283119F4877E816106C0282F217188
:1023C000213111F48E7E886194FD877E089580E02E
:1023D00008950C94530E0E94ED128FE39CE901972F
:1023E000F1F700C000000E94ED1280E00E9425126B
:1023F00080FF04C00E94E9110C94E52508950C9417
:10240000EB110E94590E811102C00E94010F0E941F
:10241000640E809365020E946C0E9093BD028093BF
:10242000BC020E94FF110E94680E682F70E080E0DD
:1024300090E00E9476086091D3017091D401809160
:10244000D5019091D6010C94AE08E82FF0E0EC5342
:10245000FD4F80810895089580EA8A95F1F70895E7
:1024600000C008950C942C1208950C9434120C940E
:1024700035120C9434120C943912F894E82FE2952A
:10248000EF70F0E031A1282F2F7081E090E001C0C3
:10249000880F2A95EAF7982F9095932391A392A1FC
:1024A000892B82A3789408950F931F93CF93DF9382
:1024B000C4E9D1E089918F3F11F00E943D1281E083
:1024C000CA39D807B9F7C0E9D1E004E911E0899128
:1024D0008F3F11F00E943D120C171D07C1F7DF91CD
:1024E000CF911F910F910895CF92DF92EF92FF92BB
:1024F0000F931F93CF93DF938C01C62FD0E0CE01B3
:102500008C569E4F7C01FC0190819F3F09F447C08F
:10251000D62EF894E92FE295EF70F0E081A19F703C
:1025200021E030E001C0220F9A95EAF7822B81A3C7
:1025300082A12095282322A378940E943012E0E9FA
:10254000F1E044E951E031E0C12C21912F3F89F0C5
:10255000A22FA295AF70B0E090968C9190E02F7072
:1025600002C0959587952A95E2F780FD02C0832FDA
:1025700001C080E0C82A330F4E175F0731F7F7011B
:1025800080818F3F11F00E943D1261E0C11001C0B7
:1025900060E08D2D0E943212C00FD11FC882DF91E2
:1025A000CF911F910F91FF90EF90DF90CF90089502
:1025B0000E94541286E0E4ECF2E0DF01982F1D92B5
:1025C0009A95E9F7EEEBF2E0DF011D928A95E9F7C3
:1025D00086E00E9435130C943F03FF920F931F93E4
:1025E000CF93DF9300D000D000D0CDB7DEB78E01FF
:1025F0000F5F1F4F86E0F80111928A95E9F7F12CE1
:102600006F2DC8010E947412F394F6E0FF12F8CF08
:1026100046E050E0B8018EEB92E00E94242DFF24AA
:10262000F394009709F4F12C892B41F086E0F8012E
:10263000AEEBB2E001900D928A95E1F72F2D46E0C6
:1026400064EC72E08EEB92E00E9436130E9441032C
:102650008F2D26960FB6F894DEBF0FBECDBFDF914B
:10266000CF911F910F91FF9008950895FF920F93BE
:102670001F93CF93DF938C01F62ED72FC42F2223E5
:1026800049F081E0809368020E9498259093670248
:1026900080936602809168028823C1F0809166026F
:1026A000909167020E94B025059780F0EF2DFD2FD5
:1026B000D8014C2F50E0CD01801B910B841795075A
:1026C0001CF48D918193F7CF10926802DF91CF9126
:1026D0001F910F91FF9008950E949B270E943E0F2B
:1026E0000C94A7270E94AB270E94D00F0C94C527FB
:1026F0000E9436250E9482270E942C0F0E946C1394
:102700000E9472130E94340FFBCF80916F0280FFF2
:1027100006C06091090170E0660F771F2CC081FF31
:1027200008C06091090170E0660F771F660F771F80
:1027300022C082FF09C06091090170E043E0660F8A
:10274000771F4A95E1F717C060916E026623D1F0BA
:1027500020910801621778F78091090190E070E0FC
:1027600033E0880F991F3A95E1F70E949D2C622F64
:1027700070E00E94DB2C6038710540F46115710532
:1027800019F406C068E070E0862F08958FE7089579
:1027900081E0089580916F0280FF08C0609105017B
:1027A00070E0759567957595679523C081FF06C0A4
:1027B0006091050170E0759567951BC082FF04C0AC
:1027C0006091050170E012C060916D026623A9F06E
:1027D000209104016217A0F78091050170E090E05C
:1027E0000E949D2C622F70E00E94DB2C60387105E6
:1027F00040F46115710519F406C061E070E0862FA0
:1028000008958FE7089581E008958D3E21F40E9498
:102810008513819504C08E3E29F40E948513809310
:10282000730208958F3E21F40E948513819504C0A0
:10283000803F29F40E948513809372020895893F96
:1028400019F40E94CA1305C08A3F31F40E94CA13CA
:1028500081958093740208958B3F21F40E94CA13DE
:10286000819504C08C3F29F40E94CA13809375029D
:1028700008959FE0980F983078F421E030E0A901A6
:1028800002C0440F551F9A95E2F7CA019091710258
:10289000892B8093710208958D3F21F480916F02FE
:1028A00081600BC08E3F21F480916F02826005C071
:1028B0008F3F29F480916F02846080936F020895A6
:1028C0008D3E39F49091730297FF35C010927302D8
:1028D00059C08E3E29F4909173021916BCF32BC097
:1028E000909172028F3E29F497FF25C010927202D8
:1028F00049C0803F19F41916CCF31DC090917402A1
:10290000893F29F41916BCF4109274023BC08A3F27
:1029100019F497FF10C0F8CF8B3F39F490917502EE
:1029200097FF09C0109275022DC08C3F21F4909141
:1029300075021916BCF39FE0980F983080F421E0DF
:1029400030E0A90102C0440F551F9A95E2F7CA0171
:1029500080959091710289238093710213C08D3FFD
:1029600021F480916F028E7F0BC08E3F21F4809105
:102970006F028D7F05C08F3F29F480916F028B7F9E
:1029800080936F0280917202811106C08091730260
:10299000811102C010926E0280917402811106C0F2
:1029A00080917502811102C010926D0208950E94FB
:1029B000982520917202211104C0209173022223D4
:1029C00021F090936C0280936B022091740221118C
:1029D00004C020917502222321F090936A02809313
:1029E000690280E792E00C940524EF92FF920F9326
:1029F0001F93CF93DF9300D000D000D0CDB7DEB7C8
:102A000086E0E0E7F2E0DE01119601900D928A95F2
:102A1000E1F7E0907202F09073020091740210915D
:102A20007502109272021092730210927402109248
:102A30007502E11003C0FF2009F464C080916B02AD
:102A400090916C020E94B025FC0120916E0222231D
:102A500039F080910A0190E08E179F0760F052C014
:102A600080910B0190E06AE070E00E949D2C8E172F
:102A70009F0718F047C02F3F19F02F5F20936E0279
:102A8000EE2061F00E948513682F1E1414F08FEF62
:102A900001C081E00E94942C80937202FF2061F0BB
:102AA0000E948513682F1F1414F08FEF01C081E07E
:102AB0000E94942C8093730280917202882311F1FA
:102AC000209173022223F1F0082E000C990B65EB84
:102AD00070E00E949D2C992319F09093720203C01C
:102AE00081E080937202822F220F990B65EB70E0D8
:102AF0000E949D2C992319F09093730203C081E0EA
:102B000080937302011103C0112309F464C0809102
:102B1000690290916A020E94B025FC0120916D0229
:102B2000222339F08091060190E08E179F0760F014
:102B300052C08091070190E06AE070E00E949D2CF5
:102B40008E179F0718F047C02F3F19F02F5F209373
:102B50006D02002361F00E94CA13682F101614F052
:102B60008FEF01C081E00E94942C809374021123A6
:102B700061F00E94CA13682F111614F08FEF01C084
:102B800081E00E94942C80937502809174028823C6
:102B900011F1209175022223F1F0082E000C990BFF
:102BA00065EB70E00E949D2C992319F090937402BC
:102BB00003C081E080937402822F220F990B65EB92
:102BC00070E00E949D2C992319F09093750203C028
:102BD00081E0809375028091720281110BC0809117
:102BE0007302811107C080917402811103C080912A
:102BF000750281110E94D714EB82FC820D831E8323
:102C000086E0FE013196A0E7B2E001900D928A9530
:102C1000E1F726960FB6F894DEBF0FBECDBFDF9169
:102C2000CF911F910F91FF90EF900895E0E7F2E0B0
:102C300086E0DF011D928A95E9F710926E021092EC
:102C40006D0210926F020895EF92FF920F931F93FF
:102C5000CF93DF93E82F71110AC0442321F0F0E0F5
:102C6000ED50FD4FE4916E2F7E2F8E2F6CC0C62F3E
:102C7000D0E0072F10E0282F30E0442329F0F9019D
:102C8000ED50FD4F249130E0CE0166E070E00E94EF
:102C90009D2CEE24EA94F12CB7010E94C72CDB0195
:102CA000CC0FDD1FCB016BEA7FEF0E949D2C8C0FB8
:102CB0009D1FC82FCC0FC80FC701801B910BB901F6
:102CC0000E949D2CE92F492FD0E0CE01B8010E942F
:102CD0009D2C692F70E0C701861B970BB9010E94DC
:102CE0009D2CF92FC7018C1B9D0BB8010E949D2CB8
:102CF000692F70E0C701861B970BB9010E949D2CBC
:102D0000A230B10591F038F4109759F01197C1F441
:102D10008E2F7F2F0CC0A430B10579F050F016979C
:102D200079F4722F842FE92F0DC0892F7E2FE22F87
:102D300009C0822F7E2FEF2F05C0822F792F02C06E
:102D4000722F8F2F6E2FDF91CF911F910F91FF90D8
:102D5000EF90089541E00E942416089508950E947E
:102D6000AA160895CF93DF93762FE901682F842F59
:102D70000E94AF16798368838A83DF91CF9108958B
:102D80008091CA02282F269530E02115310519F4CB
:102D90008170826005C02532310524F0817088641D
:102DA0008093CA02089588E090E00C94392DCF9268
:102DB000DF92EF92FF926B017C010E94C016B70177
:102DC000A60188E090E0FF90EF90DF90CF900C9408
:102DD000572DEAECF2E083E0808311828FEF82834B
:102DE0008383148260817181828193810C94D716D0
:102DF0008091CA0280FF02C08695089580E0089500
:102E00009091CE02933018F49F5F9093CE02882366
:102E100051F06091CA027091CB028091CC029091E6
:102E2000CD020C94D716089581E00C940017909170
:102E3000CE02992319F091509093CE02882351F03D
:102E40006091CA027091CB028091CC029091CD0228
:102E50000C94D716089581E00C94171770E00C9429
:102E60001C20309110018091CA0280FF0CC080911B
:102E70000F0190E063E070E00E949D2C632F81536E
:102E80009D4F0C942E17209111014091120124178F
:102E900070F7822F90E063E070E00E949D2CFC01AF
:102EA000E153FD4F1182108212822F5FF0CFA82FC5
:102EB000B62F8091CA0280FF16C020911101309177
:102EC0001201231770F4822F90E063E070E00E94FB
:102ED0009D2CFC01E153FD4FA183B08342832F5F02
:102EE000F0CF0C9431170895CF93DF9300D01F9249
:102EF000CDB7DEB79091CA0290FF0AC09E012F5F46
:102F00003F4F0E94B2164B8169818A810E945717F8
:102F10000F900F900F90DF91CF910895CF93DF9393
:102F2000EC01EC81F0E0E259FE4F4491EAECF2E072
:102F3000628181810E9474178C818F5F8C83DF9105
:102F4000CF910895CF93DF93EC01EAECF2E0438157
:102F500062818C810E9474178C818F5F8C83DF91DA
:102F6000CF9108950F931F93CF93DF9300D01F92BB
:102F7000CDB7DEB78C018091760281110AC09E0127
:102F80002F5F3F4F4FEF6FEF0E94B2168A81809301
:102F90007602F8018481813051F028F0823061F4AA
:102FA000409176020AC08091760240E007C06091AD
:102FB000760240E080E003C040E080E060E00E94F4
:102FC0005717F801848190E0019663E070E00E9459
:102FD000DB2C84830F900F900F90DF91CF911F9186
:102FE0000F910895AF92BF92CF92DF92EF92FF922E
:102FF0000F931F93CF93DF9300D01F92CDB7DEB70F
:10300000182FF62E042FE22E9091CA0290FF6EC068
:10301000E92FE695AE2FB0E0A656BE4F8C91809377
:1030200082029E7F923061F49E012F5F3F4F812F7D
:103030000E94B2164B8169818A810E94571744C051
:10304000823019F40091CD023FC0863019F41091FE
:10305000CB023AC08930D9F38931B1F5E9514E2F0D
:103060004170D42EE695F0E0E259FD4FA590B49062
:10307000C12CBB2440911301C41620F52C2D30E047
:10308000C501B9010E949D2C642F70E00E94C72CDD
:10309000E12FD11002C0E60F01C0E61B80911101A3
:1030A000A901480F511DCA0163E070E00E949D2CE8
:1030B0009C0121533D4F402F6F2D8E2F0E94B21641
:1030C000C394D8CF0E9431171093CB02F092CC0258
:1030D0000093CD02EE2051F06091CA027091CB02B4
:1030E0008091CC029091CD020E94D7160F900F9044
:1030F0000F90DF91CF911F910F91FF90EF90DF9094
:10310000CF90BF90AF900895EAECF2E09181282F24
:103110004381628188E0890F0C94F21781E00C945E
:103120008418EAECF2E09181282F4381628188EFD4
:10313000890F0C94F21781E00C949118EAECF2E0FC
:10314000628128E0620F08F46FEF282F43818181AC
:103150000C94F21781E00C949E18EAECF2E0628184
:1031600028E0621B08F460E0282F438181810C94E1
:10317000F21781E00C94AD18EAECF2E0438128E00C
:10318000420F08F44FEF282F628181810C94F217CF
:1031900081E00C94BC18EAECF2E0438128E0421B89
:1031A00008F440E0282F628181810C94F21781E0BD
:1031B0000C94CB1820E00C94F217EF92FF921F931F
:1031C000CF93DF93EC0110E0EE24EA94F12C3091E0
:1031D0001301131700F520911101812F90E0820F48
:1031E000911D63E070E00E949D2CFC01E153FD4FB6
:1031F000632F70E0C7010E94DB2C812F0E94942C6A
:103200009C819F014091CD026091CC02890F0E9468
:10321000B2161F5FDCCF0E9431179A818C8190FF1C
:1032200002C08F5F01C081508C83DF91CF911F91CD
:10323000FF90EF900895BF92CF92DF92EF92FF92AE
:103240000F931F93CF93DF93FC01828180FF02C015
:10325000DFEF01C0D1E0C0E080911301C81708F092
:1032600040C080911101CC2ED12C9601280F311D28
:10327000C90163E070E00E949D2C81539D4F7C0149
:10328000FC0111821082128204E010E0B12C8091C6
:1032900078028B0D813114F08F7005C087FF03C059
:1032A00090911301890F082E000C990BC816D906AE
:1032B00091F48091CD0290E0B8010E949D2C9595EB
:1032C0008795959587959701482F6091CC028091BD
:1032D000CB020E94B216BD0E01501109C1F6CF5F9C
:1032E000BBCF0E94311780917802D13031F4811127
:1032F00002C080911301815007C090E00196609157
:10330000130170E00E94DB2C80937802DF91CF9153
:103310001F910F91FF90EF90DF90CF90BF90089595
:10332000CF932091110130911201231770F4822F55
:1033300090E063E070E00E949D2CFC01E153FD4FA2
:103340001182108212822F5FF0CFC0E060911301D2
:10335000C61790F5EC2FF0E070E0CF010E94DB2C57
:1033600090911101890F20917702022E000C330BEE
:1033700090E063E070E00E949D2CE217F307A4F058
:1033800020910E01022E000C330B2E173F0764F024
:103390009C0121533D4F4091CD026091CC02809120
:1033A000CB020E94B21606C0FC01E153FD4F118210
:1033B00010821282CF5FCACF0E94311720910D0177
:1033C00080917702820F8093770290910E01920F85
:1033D00090930E0119165CF4082E000C990B409185
:1033E000130150E041505109841795071CF02195B5
:1033F00020930D01CF9108954F925F926F927F922B
:103400008F929F92AF92BF92CF92DF92EF92FF92F4
:103410000F931F93CF93DF938C01FC01C481CC2EBB
:10342000D12CE12CF12CA7019601C701B6010E9415
:10343000AE2CA70196010E94AE2C4B015C0180E2EC
:1034400090E06C01CC1AD1080D2C000CEE08FF089E
:1034500025E530E040E050E0C501B4010E94AE2C0B
:103460002B013C01A7019601C701B6010E94AE2CB9
:10347000A70196010E94AE2C9B01AC01280D391DBD
:103480004A1D5B1DC301B2010E94EF2CD22F822F77
:1034900090E02A3230F025E530E0A901481B590BB5
:1034A000CA0163E070E00E949D2C97FD01969595FE
:1034B0008795C82FC095F12C85E5E82EED1A8091EF
:1034C0001301F816D0F4F1FC02C0EE2D01C0ED2F6F
:1034D000209111018F2D90E0820F911D63E070E02B
:1034E0000E949D2C9C0121533D4F4C2F6091CC029A
:1034F0008E2F0E94B216F394E2CF0E943117F8018A
:103500008481811102C091E003C0803219F49FEFE1
:1035100090930C0190910C01890FF8018483DF9145
:10352000CF911F910F91FF90EF90DF90CF90BF90C0
:10353000AF909F908F907F906F905F904F90089585
:103540000F931F93CF93DF93EC0100E010E04091C5
:103550001301842F90E0081719072CF580911101B1
:103560009801280F311DC90163E070E00E949D2C75
:103570009C0121533D4F469550E08C81041715075F
:103580001CF4882331F002C0811103C04091CD02A8
:1035900001C040E06091CC028091CB020E94B21643
:1035A0000F5F1F4FD4CF0E9431178C8190E001969E
:1035B000817099278C83DF91CF911F910F9108958E
:1035C000EAECF2E080818E7F80836081718182816C
:1035D00093810E94D716109283022FEF80E792E02A
:1035E000215080409040E1F700C000000C9431175A
:1035F000EAECF2E080818E7F8083109283022FEFCD
:1036000080E792E0215080409040E1F700C0000048
:103610000C943117109283028091800281110AC0AC
:1036200081E0809380028091CA02817080937F0242
:103630000C94F81A08956091CA02669570E04BE008
:1036400050E084E191E00E94172D892B19F481E06C
:10365000809383020E94982590937A028093790246
:1036600008959091CA0290FF35C09170811102C0F7
:10367000926006C0853210F0986402C0880F982BC3
:103680009093CA02662351F06091CA027091CB02F6
:103690008091CC029091CD020E94D7166091CA020F
:1036A000669570E04BE050E084E191E00E94172DB8
:1036B000892B19F01092830202C00E941B1B81E02B
:1036C00080937C024091CD026091CC028091CB022C
:1036D0000C94DA180895682F9091CA02969581E0AB
:1036E000890F853208F081E00C94311B81E00C9445
:1036F0006B1B682F9091CA0296958FEF890F09F482
:1037000084E20C94311B81E00C94791B61E00C94F1
:10371000311BEAECF2E080818160808386950C9415
:10372000861B8091CA0280FD0C94E01A0C94891BC0
:1037300060E00C94311B8091810281112EC00E94A7
:10374000590E811104C00E94010F0E94E9160E94C7
:10375000D3166093CA027093CB028093CC029093ED
:10376000CD026E7F61F40E94E9160E94D316609329
:10377000CA027093CB028093CC029093CD020E9438
:10378000C016109283028091CA0280FF03C0869502
:103790000E94981B81E0809381020895EAECF2E098
:1037A00080818160808386950C94981B10928002A2
:1037B00080917F0281110E94CE1B0C941B1B0F93E2
:1037C0001F93CF93DF9380918302882309F485C0F0
:1037D00080918202E091CA02E695E81BE0937B02A9
:1037E000823049F4F0E0E659FE4FE491CE2FD0E06C
:1037F0000EE817E149C0863049F4F0E0E959FE4F80
:10380000E491CE2FD0E002EA17E13EC0893051F4B6
:10381000E695F0E0EC59FE4FE491CE2FD0E00DEDAF
:1038200018E132C08F3051F4E695F0E0EF59FE4FC9
:10383000E491CE2FD0E00BE119E126C0853149F4A7
:10384000F0E0E25AFE4FE491CE2FD0E000E919E11A
:103850001BC0883181F0833239F4ECE5F1E0C59189
:10386000D49102EB17E110C0843251F4C4EFD1E0DF
:1038700000EA1AE109C0C8E2D0E00CEF19E104C087
:10388000C0EDD7E00EEA16E180917C02882361F05A
:1038900010927C020E94982590937A02809379027C
:1038A00010927E0210927D020E949825E09179028A
:1038B000F0917A028E1B9F0B8F3F9F4770F4EC0FA5
:1038C000FD1FF0937A02E093790289E792E0F80114
:1038D000DF91CF911F910F910994DF91CF911F91AB
:1038E0000F910895882311F0FA0101C0FB0109949A
:1038F000CF93DF93C82FD62F0E94F8168C1740F075
:103900000E94F8168D1720F4DF91CF910C94761B4E
:103910008C2FDF91CF910C94861B1F93CF93DF9355
:10392000FB0112811111C3C0EC010E94700D827263
:10393000CD3CFCE5DF0709F49AC0A8F5C73CECE5EF
:10394000DE0709F476C0A8F4C43C9CE5D90709F465
:103950005FC028F4C33CDC4509F457C054C0C53CE3
:103960009CE5D90709F459C0C63CDC4509F45CC0A4
:103970004AC0CA3CFCE5DF0709F46AC050F4C83C01
:10398000ECE5DE0709F45AC0C93CDC4509F45BC02C
:103990003AC0CB3C9CE5D90709F45FC0CC3CDC4580
:1039A00009F460C030C0C23DFCE5DF0709F46FC018
:1039B00088F4CF3C9CE5D90709F460C008F45CC0EA
:1039C000C03DFCE5DF0709F45CC0C13DDC4509F4FE
:1039D0005BC019C0C53D9CE5D90709F460C050F42F
:1039E000C33DFCE5DF0709F455C0C43DDC4509F4DF
:1039F00054C009C0C63D9CE5D90709F455C0CE3571
:103A0000DD4509F454C011E052C00E94911B4FC023
:103A100043E85BE166E77BE104C046E75BE163E81E
:103A20007BE10E94721C43C04BE958E16EE878E1EB
:103A3000F8CF4EE858E16BE978E1F3CF49EB58E174
:103A40006AEA78E1EECF4AEA58E169EB78E1E9CF3A
:103A500047ED58E168EC78E1E4CF48EC58E167EDD8
:103A600078E1DFCF4BE257E164E177E1DACF44E17F
:103A700057E16BE277E1D5CF81E017C065E082E0E6
:103A800010C068E086E00DC06EE089E00AC064E125
:103A90008FE007C067E185E104C088E106C062E20B
:103AA00089E10E94781C03C083E20E94861B812F5B
:103AB000DF91CF911F91089586E090E00C94312D15
:103AC000682F86E090E00C94452D8091FF02847071
:103AD00089628093FF020C94601D8091FF0286959D
:103AE0008695869508958091FF0281FD07C08260CA
:103AF0008093FF020E94601D0C94631F08958091C3
:103B0000FF0281FF07C08D7F8093FF020E94601D2E
:103B10000C946F1F08958091FF0281FD0C947F1D0E
:103B20000C94731D8091FF02869581700895809199
:103B30001F0108950E94590E811104C00E94010FB7
:103B40000E94651D0E945C1D8093FF02282F269510
:103B50002695269530E02630310524F0877088625E
:103B60008093FF028091FF0280FF04C086958695B6
:103B7000869501C080E00C942C1F2091FF02822FBB
:103B8000869586958695482F50E04530510554F42A
:103B90008F5F982F990F990F990F822F8770892B1C
:103BA0008093FF028091FF0281608093FF020E9458
:103BB000601D8091FF028695869586950C942C1F3A
:103BC0008091FF02982F969596959695A1F0915E1B
:103BD000990F990F990F8770892B8093FF02887F27
:103BE00091E009F490E08091FF0290FB80F98093CE
:103BF000FF020E94601D8091FF0286958695869542
:103C00000C942C1F8091FF0280FD13C08160809373
:103C1000FF02813019F489E08093FF028091FF0256
:103C20000E94601D8091FF028695869586950C9472
:103C30002C1F08958091FF0280FF08C08E7F809323
:103C4000FF020E94601D80E00C942C1F089580915B
:103C5000FF0280FD0C941A1E0C94021E9091FF022C
:103C6000892F8695869586958F5F8F7197708630A0
:103C700038F4880F880F880F892B8093FF0202C0C9
:103C80009093FF028091FF02887F91E009F490E019
:103C90008091FF0290FB80F98093FF020E94601DDB
:103CA0008091FF028695869586950C942C1F863010
:103CB00008F085E09091FF029770282F220F220FC5
:103CC000220F922B9093FF02987F21E009F420E0CD
:103CD0009091FF0220FB90F99093FF020C942C1F0F
:103CE0000E94571E8091FF020C94601DFC01DB01B5
:103CF00012968C918823F9F0EC5BFC45E730F105D6
:103D0000D8F4EA5BFF4F0C94112D85E001C080E0F0
:103D10000E94701E80E008950E94E01DFBCF0E946B
:103D2000BD1DF8CF0E94271EF5CF0E942E1EF2CF98
:103D30000E948B1DEFCF81E00895279A2F98089558
:103D40002F9808958F929F92AF92BF92CF92DF9259
:103D5000EF92FF920F931F93CF93DF938C0180918B
:103D60008600909187006CE070E00E94C72C60177D
:103D7000710730F0C80169E070E00E94C72C5EC096
:103D80008091860090918700E0908600F0908700F7
:103D9000E0918600F0918700C6E0D0E0BE010E946D
:103DA000C72C20E030E0060F171F211D311D4801F0
:103DB000590185E0880C991CAA1CBB1C8A95D1F777
:103DC000C701BE010E94C72C6F01E12CF12CA70195
:103DD0009601260F371F411D511DC501B4010E94D8
:103DE000EF2C69017A01C0918600D0918700CA0149
:103DF000B9010E94AE2C9E0140E050E00E94AE2C22
:103E0000A70196010E94AE2CDC01CB012FE0B695F4
:103E1000A795979587952A95D1F7009186001091DF
:103E2000870020E030E0081719072A073B0728F42D
:103E30006091860070918700CB01BC01CB01DF91BE
:103E4000CF911F910F91FF90EF90DF90CF90BF9097
:103E5000AF909F908F900895CF93C82F863050F4E5
:103E6000811109C080918000877F809380000E942B
:103E7000A01E06C0C5E0809180008860809380000D
:103E8000609186007091870080E090E02C2F30E0F8
:103E900040E050E00E94AE2C25E030E040E050E0F1
:103EA0000E94EF2CB42FA32F922F8827892F9A2FAF
:103EB000AB2FBB270E94A21E90938D0080938C0095
:103EC000CF91089508951092850210928402109265
:103ED0008602EFE6F0E08081816080830895EFE65E
:103EE000F0E080818E7F80830E946D1D0C942C1FDA
:103EF0001F920F920FB60F9211240F931F932F93BF
:103F00003F934F935F936F937F938F939F93AF9361
:103F1000BF93CF93DF93EF93FF938091200191E0C4
:103F2000980F823019F0909320015BC081E080935C
:103F300020010E94971D182FC0918402D091850204
:103F400021960E94971D90E068E770E00E949D2CEA
:103F5000BC01CE010E94C72C9C01909385028093E6
:103F60008402812F90E068E770E00E949D2CBC01E4
:103F7000660F672F661F770B7195C9010E94C72CCA
:103F80006F7780918602823019F4603451F404C056
:103F9000813039F46F3729F480916F008E7F8093E0
:103FA0006F00E62FF0E0ED58FD4FC49100918600C0
:103FB000109187000E946D1D282F8C2F90E0B80172
:103FC0000E949D2C6BEF74E00E94C72CCB01622FE6
:103FD00070E00E949D2C0E94A21E90938D00809301
:103FE0008C00FF91EF91DF91CF91BF91AF919F91A5
:103FF0008F917F916F915F914F913F912F911F9181
:104000000F910F900FBE0F901F9018950E949D1E4C
:104010008AE08093800089E1809381008FEF9FEF99
:1040200090938700809386000E949A1D0E94921DA3
:1040300081110C94631F0895259A25B12F7D35B108
:1040400030624FB7F894FC01CB0163E070E00E944E
:104050009D2C8E0F9F1FE817F90789F0519168E09A
:1040600035B9000000C057FF25B9550F000000C04A
:1040700000C000C025B900C06A9591F7ECCF4FBFD2
:104080008FE594E00197F1F700C000000895CF9309
:10409000DF93EC01FB018281882309F43CC1C43029
:1040A000FDE5DF0760F4CB3F9CE5D90788F49E016E
:1040B00022503C452431310508F02EC109C0C236DA
:1040C000EDE5DE0729F0C63AFDE5DF0709F024C17A
:1040D0000E946C0E9093BD028093BC02C1318CE5AE
:1040E000D80709F4C6C008F042C0C930ECE5DE07C5
:1040F00009F49BC000F5C5308CE5D80709F485C0EC
:1041000078F4C330ECE5DE0709F478C008F07AC033
:10411000C230DC4509F0F5C08091BC028160EFC07F
:10412000C7309CE5D90709F478C008F07AC08091BF
:10413000BC028061E4C0CD30FCE5DF0709F487C034
:1041400058F4CB309CE5D90709F479C008F07BC05E
:104150008091BC0288606FC0CF30FCE5DF0709F4B6
:1041600080C008F082C08091BC02877FC8C0CE3F6B
:104170009CE5D90709F471C000F5C531FCE5DF07FE
:1041800009F485C068F4C3319CE5D90709F475C00A
:1041900008F095C00E941E088091BC028F77AFC0C6
:1041A000CC3FFCE5DF07A9F108F054C0CB3FDC456C
:1041B00009F0A7C08091BD0240C0C230EDE5DE0726
:1041C00009F489C058F4C1158DE5D80709F45AC01F
:1041D00008F069C08091BD0282602FC0C236EDE553
:1041E000DE0709F47CC0C63AFDE5DF0709F481C0AB
:1041F000C330DD4509F085C080E06EC08091BC020F
:1042000082607DC08091BC0216C08091BC02886033
:1042100076C08091BD0282604FC08091BC028062F6
:104220006EC08091BC0280646AC00E941E088091AA
:10423000BC02806864C0846062C081603DC08091BF
:10424000BC028E7F5CC08091BC028D7F58C0809183
:10425000BC0216C08091BD0218C08091BD028D7F46
:104260002BC08091BC028F7E4AC08091BC028F7DA2
:1042700046C08091BC028F7B42C08091BC02877F88
:104280008B7F3DC08091BD028D7F8E7F15C0809158
:10429000BC0282FB222720F991E0922790FB82F951
:1042A00090FB83F92CC08091BD02982F909591705E
:1042B0008E7F892B90FB81F98093BD0222C00E94E2
:1042C0001E088091BC0287FB222720F991E09227EB
:1042D00090FB87F914C081E00E94030F12C0809107
:1042E000BC0284FB222720F991E0922790FB84F9FD
:1042F00006C08091BC02982F909590FB80F9809326
:10430000BC028091BC029091BD020E947D0E0E9471
:104310001E0880E001C081E0DF91CF9108958932CD
:1043200089F1F0F4843171F1B0F4873009F077C08D
:1043300081E080930B0184E180930A018AE08093FD
:1043400009018EE18093080188E08093050188E2ED
:104350008093040164C092EE980F9A30F0F05FC031
:10436000803509F444C028F48F3409F058C08AE03D
:104370003FC0813529F0823509F051C081E038C055
:104380008FEF36C080918902882379F110928902DB
:10439000109288021092870242C08D518093890248
:1043A000833099F038F4813069F08230D9F48AE0B2
:1043B00091E00DC0853099F078F0863099F484E072
:1043C00091E005C08BE091E002C089E091E090931C
:1043D00088028093870223C088E091E0F8CF85E0CF
:1043E00091E0F5CF109289021AC080E0089586EF1F
:1043F000E0918702F0918802309789F02081082EA1
:10440000000C990B820F911D8F3F910519F014F04C
:104410008FEF04C097FF02C0108201C0808381E04B
:1044200008950F931F9341E050E060E070E08A012F
:104430009B0104C0000F111F221F331F8A95D2F762
:10444000C901B8010E9476081F910F910C941E08B3
:10445000482F50E0FA013597EF33F10508F060C0BE
:10446000E35BFF4F0C94112D0E94010F55C080910A
:104470006502817F8E7F8093650281E080938A024E
:1044800008950E94440348C080916502982F90953A
:10449000917090FB80F98093650291113DC0897FF6
:1044A000877F10C08091650281FB222720F991E06F
:1044B000922790FB81F980936502992369F180919D
:1044C000650281608093650227C08091650282FB4E
:1044D000222720F991E0922790FB82F9ECCF80917E
:1044E000650283FB222720F991E0922790FB83F954
:1044F000E2CF0E941E088091BC0287FB222720F990
:1045000091E0922790FB87F98093BC0205C0895304
:1045100001C08D510E94112281E0089580E0FACF00
:1045200080E0089580E008950C949222CF93C82FE4
:1045300080918A02813069F038F08230C1F58C2F89
:104540000E948F2181E039C00E94700D823289F56E
:1045500004C00E94700D823261F48C2F0E9494225C
:10456000811104C08C2F0E9428221FC081E090E09E
:104570001CC08C2F0E949222811116C0C43189F078
:1045800058F4CB3089F0C031B1F482E080938A02D4
:1045900088E30E948F2108C0C93219F0C83321F086
:1045A0000AC010928A0207C081E0817006C0109292
:1045B0008A0280E002C080E0F8CFCF910895CF93C7
:1045C000DF9386319C4541F5EB010E94700D982FD9
:1045D0008A812091020130910301882379F09A7A2F
:1045E00081E009F480E080938B02911102C069E2BE
:1045F00001C065E3C9010E94D5240AC080918B02E5
:10460000811102C069E201C065E3C9010E94E02492
:104610000E94B20D80E001C081E0DF91CF9108954A
:104620000F931F93CF93DF93C42FD22FFC0182816E
:104630008823C9F040938E020E94982590938D02A2
:1046400080938C0280E28C0F883008F057C0C770CE
:1046500081E001C0880FCA95EAF7DF91CF911F91E1
:104660000F910C947B0580918E02481330C080918D
:104670008C0290918D020E94B025883C910538F5FE
:1046800010E21D0FCD17B9F080E28C0F883040F496
:10469000C77081E001C0880FCA95EAF70E948205C1
:1046A000183028F581E09D2F977001C0880F9A95EA
:1046B000EAF70E947B05802F0E9472051830F0F403
:1046C000D77081E001C0880FDA95EAF70AC080E26E
:1046D0008C0F883098F4C77081E001C0880FCA95AC
:1046E000EAF7DF91CF911F910F910C948205802FF3
:1046F000DF91CF911F910F910C947205DF91CF91B3
:104700001F910F9108950F939C01CB01243F4CE51D
:10471000340731F188F4293DFCE53F07D9F02A3D03
:104720004CE5340779F1283D3C45A9F506E221EE38
:1047300041EE68ED7CE52BC0263FFCE53F07E1F04C
:10474000A8F0273F3C4539F507E225EE46EE67EF36
:104750007CE51DC007E225EE45EE69ED7CE517C05E
:1047600006E221EE40EE64EF7CE511C007E225EEA3
:1047700044EE65EF7CE50BC006E221EE42EE66EF0B
:104780007CE505C008E221E045EE6AED7CE50E948B
:10479000102380E008C0FC018281882319F0109268
:1047A0008E0201C081E00F9108959093C101809322
:1047B000C001089590939402809393020895E0912C
:1047C0009302F0919402309721F00190F081E02D56
:1047D000099480E00895E0919302F091940230975B
:1047E00099F020912D01222359F02091BC0227FF3E
:1047F00007C0DC012C9111962C93119726E02C9385
:104800000280F381E02D09940895E0919302F091E4
:104810009402309739F022E0DC012C930480F5817A
:10482000E02D099408952091910230919202281769
:10483000390771F09093920280939102E091930274
:10484000F0919402309721F00680F781E02D0994D1
:10485000089520918F02309190022817390771F046
:104860009093900280938F02E0919302F0919402D2
:10487000309721F00084F185E02D09940895FC0122
:10488000329680912D01882331F08091BC0287FF00
:1048900002C09EE101C096E080E0915028F0219195
:1048A0002223D9F38F5FF9CF0895662351F1209128
:1048B0002D012223E9F02091BC0227FF19C0462FC9
:1048C0004695469546954E31E0F4677021E030E01C
:1048D00002C0220F331F6A95E2F7FC01E40FF11DBD
:1048E000828190E02823392381E0232B69F409C0D9
:1048F000FC01329608962191621729F0E817F90712
:10490000D1F780E0089581E008959C01FC01329682
:104910009FEF80E04191461789F09F3F19F44111C4
:1049200001C0982F8F5F8630A9F79F3F39F0F901BA
:10493000E90FF11D97FDFA956283089508959C0192
:104940002A5F3F4FFC014281461301C0128201964B
:1049500082179307B9F70895262F26952695269551
:104960002E3168F4FC01E20FF11D677021E030E0A8
:1049700001C0220F6A95EAF78281282B22830895CD
:10498000262F2695269526952E3170F4FC01E20FF0
:10499000F11D677021E030E001C0220F6A95EAF74F
:1049A0002095828128232283089520912D0122239E
:1049B00029F02091BC0227FD0C94AC240C94852492
:1049C00020912D01222329F02091BC0227FD0C9477
:1049D000C0240C949F2420912D01FC0132962223A7
:1049E00031F08091BC0287FF02C08EE101C086E0F9
:1049F000DF011D928A95E9F7089508950C94FD242E
:104A000083E0809395020C94FE24811102C081E022
:104A100001C082E0809395020C94FE240C9405253D
:104A200081E0809395020C94FE240C941025089547
:104A30000C9417250C9418250C9417250C94172505
:104A40000C941725CF930E941E250E94ED120E9400
:104A50001C25C0E08C2F0E942512811104C0CF5F5D
:104A6000C630C1F701C081E0CF91089508951F922B
:104A70000F920FB60F9211248F939F93AF93BF9312
:104A800080919602811113C08091000390910103DF
:104A9000A0910203B09103034196A11DB11D809323
:104AA000000390930103A0930203B0930303BF910B
:104AB000AF919F918F910F900FBE0F901F901895FF
:104AC00080910803843031F10E94B3031092960262
:104AD00020E488E190E00FB6F894A89580936000F8
:104AE0000FBE2093600083B7817F846083BF83B74C
:104AF000816083BF7894889583B78E7F83BF0FB61C
:104B0000F894A8958091600088618093600010926D
:104B100060000FBE08950E941E080C94BC0382E042
:104B200084BD93E095BD9AEF97BD80936E00089584
:104B30002FB7F8948091000390910103A091020394
:104B4000B09103032FBF08952FB7F894609100032D
:104B50007091010380910203909103032FBF089588
:104B60009C014FB7F8948091000390910103A091AC
:104B70000203B09103034FBF821B930B08957894F7
:104B80001F920F920FB60F9211248F939F93AF93A2
:104B9000BF938091000390910103A0910203B09113
:104BA00003030196A11DB11D80930003909301039F
:104BB000A0930203B0930303BF91AF919F918F9194
:104BC0000F900FBE0F901F90189581E08093E0002A
:104BD00080E28093D8001092C9008FE19EE4019793
:104BE000F1F700C0000087E090EBDC018093110337
:104BF00090931203A0931303B09314039CE088E1F5
:104C00000FB6F894A895809360000FBE9093600053
:104C1000FFCF8091BA020895089522E02093E90021
:104C20002FEF3091E800215035FD06C035ED3A9563
:104C3000F1F700002111F5CF2091E80025FF0BC00E
:104C400040E050E066E070E00E9437288091E80084
:104C50008E778093E8000895CF93DF9320912D0104
:104C6000222339F02091BC0227FF03C060E222E03A
:104C700002C068E021E02093E9002FEF3091E800C6
:104C8000215035FD06C035ED3A95F1F700002111B0
:104C9000F5CF2091E80025FF1DC0EC0180912D018A
:104CA000811105C040E050E068E070E003C070E0B2
:104CB00040E050E0CE010E9437288091E8008E77D6
:104CC0008093E80080E2FE01AAE9B2E001900D9233
:104CD0008A95E1F7DF91CF910895809397027093C1
:104CE00099026093980280910803843001F582E074
:104CF0008093E9008FEF9091E800815095FD06C008
:104D000095ED9A95F1F700008111F5CF8091E800BB
:104D100085FF0DC040E050E063E070E087E992E07D
:104D20000E9437288091E8008E778093E8000895EC
:104D3000BC0184E00C946D26BC0183E00C946D26CC
:104D40000C9415256091040381E0611101C080E09D
:104D50000C9400259091080381E0943009F080E0E4
:104D6000609104030C94052542E061EC81E00E940F
:104D70003B2942E261EC82E00E943B2990910803CA
:104D800081E0943009F080E0609104030C940E25DA
:104D900080910A03833009F45DC030F4813071F0F2
:104DA000823009F496C008958A3009F482C08B30AD
:104DB00009F468C0893009F0A4C020C080910903BB
:104DC000813A09F09EC08091E800877F8093E800D7
:104DD00080910D0390910E03892B21F460E28AE902
:104DE00092E003C060E080E090E070E00E948228E2
:104DF0008091E8008B778093E80008958091090303
:104E0000813209F07EC080910D0390910E030297CC
:104E100008F077C08091E800877F8093E800809158
:104E2000E80082FD05C0809108038111F8CF69C0B8
:104E30008091F200823031F48091F100813011F0E4
:104E4000863021F48091F1008093BA028091E800CD
:104E50008B7753C080910903813A09F052C0809149
:104E60000D0390910E03892B09F04BC08091E8004F
:104E7000877F8093E8008091E80080FFFCCF8091DD
:104E80002D0136C0809109038132D9F580910D033F
:104E900090910E03892BA9F58091E800877F80937C
:104EA000E8000E94702980910B0380932D010C94DF
:104EB0001E0880910903813221F58091E800877FE7
:104EC0008093E8000E94702980910C038093BB02BC
:104ED000089580910903813AA1F48091E800877FC9
:104EE0008093E8008091E80080FFFCCF8091BB02B6
:104EF0008093F1008091E8008E778093E8000C9415
:104F00007029089584B7877F84BF0FB6F894A89559
:104F100080916000886180936000109260000FBEF5
:104F200090E080E80FB6F894809361009093610060
:104F30000FBE0C9410250E94C2290E94152AE2EE91
:104F4000F0E080818460808378940C94792C81E2F5
:104F500091E00C94DA23809108038530A9F48091C4
:104F60000803853079F40E94602580910603882328
:104F7000B1F30E942225882391F30E9421280E94E8
:104F80001E08EDCF0C948B25089508950C94C82726
:104F9000292F332723303105C9F060F42130310542
:104FA00081F02230310509F044C08BE390E023E228
:104FB00034E043C021323105E1F02232310549F1BC
:104FC00038C082E190E02EE534E037C09927813087
:104FD000910549F028F0029761F5E3EFF3E005C091
:104FE000EFE1F4E002C0EDE0F4E0849190E09F0195
:104FF00024C06115710541F061307105D1F489E07B
:1050000090E02EE434E019C089E090E025E334E03C
:1050100014C06115710541F06130710551F486EBE2
:1050200090E020E734E009C080E490E026E235E03B
:1050300004C080E090E020E030E0FA01318320837A
:10504000089584E089BD86E089BD09B400FEFDCFE6
:105050008091D8008F7D8093D8008091E00082609D
:105060008093E0008091E00081FDFCCF0895CF9215
:10507000DF92EF92FF920F931F93CF93DF93EC0198
:105080008B017A010E948F29811133C0E114F10450
:1050900039F0F70180819181081B190BC80FD91FC6
:1050A000C12CD12C0115110519F18091E80085FD65
:1050B00016C08091E8008E778093E800E114F10437
:1050C00049F0F70180819181C80ED91ED182C0823A
:1050D00085E00FC00E948F29882321F30AC089919F
:1050E0008093F10001501109FFEFCF1ADF0ADACFE8
:1050F00080E0DF91CF911F910F91FF90EF90DF90B3
:10510000CF90089520910F03309110032617370791
:1051100048F06115710539F42091E8002E7720934D
:10512000E80001C0B901FC0120E06115710561F1E1
:10513000809108038823D9F18530D9F18091E80066
:1051400083FD39C08091E80082FD2BC08091E8008A
:1051500080FFEBCF8091F20090E06115710551F076
:105160008830910538F421912093F1006150710944
:105170000196F3CF21E0089709F020E08091E80044
:105180008E778093E800D1CF2111D2CF0AC08091D1
:105190000803882361F0853061F08091E80083FD89
:1051A0000AC08091E80082FFF2CF80E0089582E09B
:1051B000089583E0089581E0089520910F033091D0
:1051C00010032617370748F06115710539F420914F
:1051D000E8002E772093E80001C0B901FC0120E02F
:1051E0006115710579F180910803882309F43DC0A8
:1051F000853009F43CC08091E80083FD3AC080917D
:10520000E80082FD2CC08091E80080FFE9CF80910A
:10521000F20090E06115710559F08830910540F475
:1052200024912093F1003196615071090196F2CFDB
:1052300021E0089709F020E08091E8008E778093C4
:10524000E800CECF2111CFCF0AC080910803882378
:1052500061F0853061F08091E80083FD0AC08091A3
:10526000E80082FFF2CF80E0089582E0089583E0B5
:10527000089581E00895982F953068F59093E9009E
:10528000981739F07091EC002091ED005091F000EA
:1052900003C0242F762F50E021FD02C09F5FECCF8A
:1052A0003091EB003E7F3093EB003091ED003D7F7D
:1052B0003093ED003091EB0031603093EB00709350
:1052C000EC002093ED005093F0002091EE0027FDBC
:1052D000E5CF80E008958F708093E90081E0089524
:1052E0008091090387FF11C08091E80082FD05C00D
:1052F000809108038111F8CF11C08091E8008B776D
:105300000BC080910803882349F08091E80080FF5A
:10531000F8CF8091E8008E778093E800089520917F
:10532000E4003091E50095E64091EC00842F817017
:1053300040FF23C08091E80080FD1DC080910803DC
:10534000882399F0853099F08091EB0085FD11C09C
:105350004091E4005091E5002417350729F391505E
:1053600011F09A01E1CF84E0089582E0089583E08E
:10537000089581E0089580E008954091E80042FF9B
:10538000DDCF08950E941F2A0E94222AE0EEF0E05D
:10539000808181608083E8EDF0E080818F77808379
:1053A00019BCE3E6F0E080818160808310920703FE
:1053B00008950E941F2A0E94222A8091D8008F7788
:1053C0008093D8008091D80080688093D800809125
:1053D000D8008F7D8093D80084E089BD86E089BDA8
:1053E00009B400FEFDCF109208031092040310923E
:1053F00006031092050342E060E080E00E943B2932
:105400008091E1008E7F8093E1008091E2008160D5
:105410008093E2008091E20088608093E2008091B6
:10542000E0008E7F8093E0000895E3E6F0E0808165
:105430008E7F808381E0809307030C94D92910929A
:10544000E20008951092E10008951F920F920FB6A6
:105450000F9211242F933F934F935F936F937F93FA
:105460008F939F93AF93BF93EF93FF938091E1004E
:1054700082FF0BC08091E20082FF07C08091E100B3
:105480008B7F8093E1000E94782C8091E10080FF67
:1054900019C08091E20080FF15C08091E2008E7FEC
:1054A0008093E2008091E20080618093E20080912D
:1054B000D80080628093D80019BC85E080930803EF
:1054C0000E94A2268091E10084FF30C08091E2001A
:1054D00084FF2CC084E089BD86E089BD09B400FE4C
:1054E000FDCF8091D8008F7D8093D8008091E1001E
:1054F0008F7E8093E1008091E2008F7E8093E200B6
:105500008091E20081608093E2008091040388230F
:1055100011F084E007C08091E30087FD02C081E0C4
:1055200001C083E0809308030E94AA268091E100D5
:1055300083FF29C08091E20083FF25C08091E100B4
:10554000877F8093E10082E0809308031092040338
:105550008091E1008E7F8093E1008091E2008E7F58
:105560008093E2008091E20080618093E20042E05B
:1055700060E080E00E943B298091F0008860809389
:10558000F0000E94A026FF91EF91BF91AF919F91F3
:105590008F917F916F915F914F913F912F910F90DC
:1055A0000FBE0F901F9018951F920F920FB60F927B
:1055B00011242F933F934F935F936F937F938F9318
:1055C0009F93AF93BF93CF93DF93EF93FF93C091DC
:1055D000E900CF708091EC00D82FD17080FDD0E829
:1055E0001092E9008091F000877F8093F00078941A
:1055F0000E94182B1092E9008091F000886080933F
:10560000F000CD2BCF70C093E900FF91EF91DF91B7
:10561000CF91BF91AF919F918F917F916F915F914A
:105620004F913F912F910F900FBE0F901F901895A3
:105630001F93CF93DF93CDB7DEB7AA970FB6F89439
:10564000DEBF0FBECDBFE9E0F3E08091F1008193B2
:1056500023E0E131F207C9F70E94C8268091E800F3
:1056600083FF2EC18091090390910A03492F50E0D6
:105670004A30510508F024C1FA01E457FF4F0C9459
:10568000112D803821F0823809F01AC108C08091AC
:10569000050390910603992389F082600FC08091E1
:1056A0000D038F70853008F00BC18093E900809165
:1056B000EB0085FB882780F91092E9009091E800C3
:1056C000977F9093E8008093F1001092F100D1C091
:1056D000282F2D7F09F0F4C0882319F0823061F063
:1056E000EFC080910B03813009F0EAC0933009F0DC
:1056F00080E0809306032EC080910B0381112AC0A5
:1057000080910D038F702FEF280F243008F0D8C040
:105710008093E9002091EB0020FF1CC0933021F41E
:105720008091EB00806214C09091EB0090619093A7
:10573000EB0021E030E0A90102C0440F551F8A951B
:10574000E2F74093EA001092EA008091EB00886053
:105750008093EB001092E9008091E800877F8093AE
:10576000E8000E947029ACC08111AAC010910B03FF
:105770001F778091E3008078812B8093E3008091F4
:10578000E800877F8093E8000E9470298091E800FC
:1057900080FFFCCF8091E30080688093E3001111CB
:1057A00002C082E001C083E08093080389C0805872
:1057B000823008F085C080910B0390910C038C3DE2
:1057C00053E0950779F583E08A838AE289834FB7AE
:1057D000F894DE01139620E03EE051E2E32FF0E082
:1057E00050935700E49120FF03C0E295EF703F5FB4
:1057F000EF708E2F90E0EA3010F0C79601C0C0968F
:105800008D939D932F5F243149F74FBF8091E8001E
:10581000877F8093E8006AE270E0CE0101960E94E3
:10582000822816C060910D0370910E03AE014F5F88
:105830005F4F0E94C627BC01892B09F441C090919B
:10584000E800977F9093E80089819A810E94DD2883
:105850008091E8008B778093E80032C0803881F532
:105860008091E800877F8093E80080910403809313
:10587000F1008091E8008E7772CF811121C0809174
:105880000B0390910C0399270297D4F48091E800C0
:10589000877F8093E80080910B03809304030E942C
:1058A000702980910403811106C08091E30087FD77
:1058B00002C081E001C084E0809308030E94B42606
:1058C0008091E80083FF0AC08091E800877F809381
:1058D000E8008091EB0080628093EB00AA960FB6FF
:1058E000F894DEBF0FBECDBFDF91CF911F91089519
:1058F0000895CF93809108038823A1F0C091E90017
:10590000CF709091EC00892F817090FD80E8C82BBA
:105910001092E9008091E80083FD0E94182BCF705F
:10592000C093E900CF910895002480FD060E660F14
:1059300011F08695D1F7802D08950024552704C0D5
:10594000080E591F880F991F009729F076956795C3
:10595000B8F37105B9F7802D952F0895EE27FF272D
:10596000AA27BB2708C0A20FB31FE41FF51F220FF1
:10597000331F441F551F969587957795679598F324
:105980007040A9F7009799F7BD01CF010895AA1BB0
:10599000BB1B51E107C0AA1FBB1FA617B70710F01A
:1059A000A61BB70B881F991F5A95A9F7809590954C
:1059B000BC01CD01089597FB072E16F4009407D083
:1059C00077FD09D00E94C72C07FC05D03EF49095C6
:1059D00081959F4F0895709561957F4F0895A1E23D
:1059E0001A2EAA1BBB1BFD010DC0AA1FBB1FEE1F59
:1059F000FF1FA217B307E407F50720F0A21BB30BA4
:105A0000E40BF50B661F771F881F991F1A9469F71F
:105A100060957095809590959B01AC01BD01CF017B
:105A20000895EE0FFF1F0590F491E02D0994FC01FD
:105A30004150504030F001900616D1F73197CF0118
:105A40000895882799270895FB01DC0104C08D91F2
:105A50000190801921F441505040C8F7881B990BE0
:105A60000895F999FECF92BD81BDF89A992780B526
:105A70000895A6E1B0E044E050E00C946B2DA8E15D
:105A8000B0E042E050E00C946B2D262FF999FECF48
:105A900092BD81BDF89A019700B4021639F01FBA81
:105AA00020BD0FB6F894FA9AF99A0FBE089503969E
:105AB000272F0E94462D0E94452D252F0E94462DFE
:105AC000242F0C94462D0196272F0E94462D0C94CE
:105AD000452DDC01CB01FC01F999FECF06C0F2BDDA
:105AE000E1BDF89A319600B40D9241505040B8F79C
:065AF0000895F894FFCFB9
:105AF600C8003502280850011E0A140101010200DF
:105B06001000101001191A1B1C1D1E1F2021220631
:105B16000109262C260D269C2698260C2601E20035
:105B2600E900EA00B500B600B700CD008301CC005D
:105B36008A019201940121022302240225022602EF
:105B460027022A02B300B4006F007000818283E24C
:105B560000E900EA00B500B600B700CD008301CC2D
:105B6600008A0192019401210223022402250226C1
:105B76000227022A02B300B4006F007000818283FC
:105B8600646533329391926667360001020202021F
:105B96000606060909090909090F0F0F0F0F0F1548
:105BA600151518191919191919191919192324006C
:00000001FF
